:100000000C9463010C9480010C9480010C94800189
:100010000C9480010C9480010C9480010C9480015C
:100020000C9480010C94D40A0C9454090C94A70AE3
:100030000C94200A0C944D0A0C9427090C94F30993
:100040000C94C8080C9480010C9409110C94800144
:100050000C94BF100C94CE010C9480010C94800180
:100060000C947A0A0C94880B0C94010B0C942E0BB4
:100070000C945B0B0C94C6090C942E110C9480010B
:100080000C94E4100C94390D0C9480012F6572725D
:100090006F722F6D73676C656E6774682F002F65C4
:1000A00072726F722F74797065746167322F002FCE
:1000B0006572726F722F74797065746167332F0087
:1000C0002F6572726F722F74797065746167342F47
:1000D000002F6572726F722F6D736773697A652F67
:1000E000002F6572726F722F636865636B73756D35
:1000F0000000000100080020004000800000010016
:10010000040000010008004000000100043031320A
:1001100033343536373839414243444546002F623F
:10012000746E31002F62746E32002F62746E330071
:100130002F62746E34002F62746E35002F62746EFD
:1001400036002F62746E37002F62746E38002F7382
:10015000777431002F736C6431002F6B6E62310045
:100160002F6164786C312F78002F6164786C312FA7
:1001700079002F6164786C312F7A002F61646335C8
:10018000002F61326432002F61646331002F656E8D
:100190006331002F736C6432002F6B6E6232002F5C
:1001A000736C6433002F6B6E6233002F736C643496
:1001B000002F6B6E6234002F61646332002F616424
:1001C0006333002F6C656431002F6C656432002F3F
:1001D0006C656433002F6C656434002F6C65643586
:1001E000002F6C656436002F736572766F31002FB7
:1001F000696E30002F696E31002F696E32002F69F1
:100200006E33002F696E34002F696E35002F696ED2
:1002100036002F696E37002F646973636F6E6E65E9
:100220006374002F636F6E6E656374002F6469736F
:10023000636F6E6E656374002F636F6E6E656374BB
:10024000002F72657363616E002F70776D002F6FE2
:100250007574002F61646330002F61646331002F77
:1002600061646332002F61646333002F616463341F
:10027000002F61646335002F61646336002F616471
:100280006337002F696E31002F696E32002F696E5F
:1002900033002F696E34002F7266696431002F724B
:1002A00066696432002F7266696433002F72666972
:1002B0006434002F61646331002F61646332002F66
:1002C00061646333000011241FBECFEFD0E1DEBFB5
:1002D000CDBF11E0A0E0B1E0EAE5F9E300E00BBF3B
:1002E00002C007900D92A230B107D9F718E0A2E042
:1002F000B1E001C01D92AD32B107E1F70C94BD1A17
:100300000C94000096B1987F982B96B9089527B168
:100310002F73992736E0880F991F3A95E1F7282B1C
:1003200027B90895379A359886E00E94820181E0C6
:100330000E9487013D98339A1092F50678940895AB
:1003400033983798089597B1907E8F71982B97B90D
:100350000895349A369A089586B1992780749070DA
:1003600008951092F50697B1907E8F71982B97B9EA
:10037000349A369A3699FECF84B1282F332785B127
:100380009927982F8827822B932B08950E94B101DB
:100390009695879596958795992708951F920F9220
:1003A0000FB60F9211248F938FEF8093F5068F91E4
:1003B0000F900FBE0F901F9018950E94E30E40E023
:1003C00052EC61E070E080E00E94A80E0895992749
:1003D00081309105A1F0823091051CF4892B21F028
:1003E00032C0029729F12FC080E00E94430F6CE2D7
:1003F0000E94B61180E00E94430F69E62EC080E0A3
:100400000E94430F6CE20E94B61180E00E94430FED
:1004100069E60E94B61180E00E94430F69E60E94DF
:10042000B61180E00E94430F60E00E94B61108956B
:1004300080E00E94430F6CE20E94B61180E00E94AF
:10044000430F63E70AC080E00E94430F6CE20E9402
:10045000B61180E00E94430F6EE40E94B61180E066
:100460000E94430F60E0DBCF0F931F93CF93DF9386
:10047000EC0100E0FE012196149180E00E94430F00
:10048000612F0E94B6110F5F1123A1F7802F9927CA
:1004900083709070892B69F080E00E94430F60E0C8
:1004A0000E94B6110F5F802F992783709070892B5F
:1004B00099F7DF91CF911F910F9108951F93CF93DB
:1004C000DF93EC01162F80E00E94430F6EEB0E9439
:1004D000B61120E0FE018491882329F02F5FFE01F0
:1004E000E20FF11DF8CF2F5F822F99278370907054
:1004F000892B11F02C7F2C5F120F80E00E94430F9C
:10050000612F0E94B611DF91CF911F9108950F9333
:100510001F93CF93DF93EC0100E0199180E00E94DC
:10052000430F612F0E94B6110F5F1123B1F7802F87
:10053000992783709070892B69F080E00E94430FA7
:1005400060E00E94B6110F5F802F99278370907032
:10055000892B99F7DF91CF911F910F9108950F93F8
:100560001F93CF93DF9300E012E008C080E00E9469
:10057000430FBE010E94A411080F1F5FC12FDD278A
:1005800080E00E94430FFC0184819581C817D90740
:1005900068F380E00E94430F602F0E94B611DF9144
:1005A000CF911F910F9108950F931F93CF93DF93D6
:1005B0008C01EB0160E0FE018491882329F06F5FDC
:1005C000FE01E60FF11DF8CF6F5F862F992783702C
:1005D0009070892B11F06C7F6C5F6C5FC8010E947A
:1005E0005E02C8010E94340282E00E94E701CE014F
:1005F0000E9434020E94AF0280E00E94F90F8091B5
:100600001F078823E1F3DF91CF911F910F91089588
:100610000F931F93CF93DF938C01EB0160E08881F0
:10062000882331F06F5FFE01E60FF11D8081F8CF66
:100630006F5F862F992783709070892B11F06C7FE4
:100640006C5F6C5FC8010E945E02C8010E943402A8
:1006500082E00E94E701CE010E9487020E94AF0261
:1006600080E00E94F90F80911F078823E1F3DF915A
:10067000CF911F910F910895EF92FF920F931F93C7
:10068000CF93DF93CDB7DEB728970FB6F894DEBFD0
:100690000FBECDBF7C0149835A836B837C830D835E
:1006A0001E832F8338876CE00E945E02C7010E9480
:1006B000340281E00E94E70180E00E94430F6C81D8
:1006C0000E94B61180E00E94430F6B810E94B61118
:1006D00080E00E94430FFE01319661810E94B611B5
:1006E00080E00E94430F69810E94B61180E00E9461
:1006F000430F68850E94B61180E00E94430F6F810E
:100700000E94B61180E00E94430F6E810E94B611D4
:1007100080E00E94430F6D810E94B6110E94AF02DB
:1007200080E00E94F90F80911F078823E1F328964B
:100730000FB6F894DEBF0FBECDBFDF91CF911F91F2
:100740000F91FF90EF9008950F931F93CF93DF9336
:10075000CDB7DEB724970FB6F894DEBF0FBECDBF7E
:100760008C0149835A836B837C8368E00E945E021C
:10077000C8010E94340280E00E94E70180E00E94EC
:10078000430F6C810E94B61180E00E94430F6B8181
:100790000E94B61180E00E94430FFE0131966181F4
:1007A0000E94B61180E00E94430F69810E94B61139
:1007B0000E94AF0280E00E94F90F80911F078823FA
:1007C000E1F324960FB6F894DEBF0FBECDBFDF91E4
:1007D000CF911F910F9108950F931F938C0160E0AB
:1007E0000E945E02C8010E9434020E94AF0280E0B3
:1007F0000E94F90F80911F078823E1F31F910F9149
:1008000008951092020110920407109202071092AC
:100810000A071092090710924401109243011092A6
:10082000030740E450E063E071E086EF96E00E9449
:100830005311E3E0F1E08FE31192815087FFFCCF89
:100840000895909344018093430108950F931F935B
:10085000282F8091020199278830910509F4C6C09C
:1008600089309105C4F48230910509F44BC083307E
:1008700091052CF4009751F1019769F1B4C18630CC
:10088000910509F440C1873091050CF09EC1059790
:1008900009F451C1A8C18C30910509F450C08D30C4
:1008A000910544F48A30910509F4E3C00B970CF0EC
:1008B00008C1B8C08E30910509F46AC08E30910528
:1008C0000CF44CC00F9709F47AC08DC12E3B09F08F
:1008D0008CC181E02DC120930407109202072F33B1
:1008E00010F482E025C1822F9927AA27BB278C010B
:1008F0009D014FE350E060E070E08CE890E00E94E2
:100900003C0344C080910207222349F0E82FFF27CF
:10091000ED5FFE4F20838F5F8093020766C1E82F53
:10092000FF27ED5FFE4F20838F5F8093020799279B
:1009300083709070892B09F058C18CE0F9C08091C8
:100940000207E82FFF27ED5FFE4F20838F5F809324
:1009500002072C3209F054C08DE0EAC080910207F2
:10096000E82FFF27ED5FFE4F20838F5F8093020704
:10097000293611F48EE0DCC0822F9927AA27BB27E5
:10098000AC01BD018EE990E00E94A40387E0D0C0D5
:1009900080910207E82FFF27ED5FFE4F20838F5FD6
:1009A00080930207222311F48FE0C2C0822F99277F
:1009B000AA27BB27AC01BD018FEA90E0E5CF80916B
:1009C0000207E82FFF27ED5FFE4F20838F5F8093A4
:1009D0000207222311F488E0ABC0822F9927AA27AF
:1009E000BB27AC01BD0180EC90E0CECF8091020727
:1009F000E82FFF27ED5FFE4F20838F5F8093020774
:100A0000822F9927AA27BB27B82FAA27992788279B
:100A10008093050790930607A0930707B0930807F4
:100A200089E086C080910207E82FFF27ED5FFE4F27
:100A300020838F5F80930207822F9927AA27BB27E5
:100A4000AC01332722278091050790910607A091DA
:100A50000707B0910807822B932BA42BB52B80930B
:100A6000050790930607A0930707B09308078AE04D
:100A70005FC080910207E82FFF27ED5FFE4F2083C4
:100A80008F5F80930207822F9927AA27BB272227EF
:100A9000382F492F5A2F8091050790910607A09172
:100AA0000707B0910807822B932BA42BB52B8093BB
:100AB000050790930607A0930707B09308078BE0FC
:100AC00037C080910207E82FFF27ED5FFE4F20839C
:100AD0008F5F8093020733274427552780910507AE
:100AE00090910607A0910707B0910807822B932BDE
:100AF000A42BB52B8093050790930607A0930707B7
:100B0000B093080714C080910207E82FFF27ED5F1C
:100B1000FE4F2083E82FEF5FE093020780910407E8
:100B2000E81709F062C0FF27ED5FFE4F108285E0F5
:100B3000809302015AC080910207409104078417F4
:100B400059F09927AA27BB275527662777278C01B5
:100B50009D0181ED90E036C01092030790E094175C
:100B600050F4392FE3E0F1E0942F8191380F915048
:100B7000E1F730930307809103078217C1F4809156
:100B8000430190914401892B71F180910507909167
:100B90000607A0910707B0910807E0914301F09183
:100BA0004401AC01BD0183E091E009951CC0992787
:100BB000AA27BB27422F5527662777278C019D013F
:100BC00081EE90E00E943C030EC0809102078F5F8F
:100BD00080930207282F33278091040799270196D5
:100BE0002817390711F4109202011F910F910895EF
:100BF0001F93182F65E480E00E944C0F612F80E066
:100C00000E944C0F812F0E9426041F910895039685
:100C100065E070E00E945C1CCB01AA27BB2724E0A2
:100C2000880F991FAA1FBB1F2A95D1F7009711F0B3
:100C30000197FCCF08958E3040F4E82FFF27EE0F88
:100C4000FF1FEB5BFE4F108211820895089593B74A
:100C5000987F982B93BF089510920B0710920C0762
:100C600010920D0710920E0710921B0710921C078E
:100C700010921D0710921E07089584E00E94270617
:100C800012BE87B7816087BF0E942C0608959EB56B
:100C9000987F982B9EBD089584E00E9447061DBC56
:100CA0001CBC87B7846087BF089595B5987F982B43
:100CB00095BD089510921707109218071092190702
:100CC00010921A0710920F07109210071092110736
:100CD00010921207089582E00E94550614BC87B74F
:100CE000806487BF0E945A06089590918A00987F79
:100CF000982B90938A00089584E00E9475061092C4
:100D000089001092880080917D00846080937D002E
:100D10000895CF93C0E08C2F0E941B06CF5FCE308A
:100D2000D0F30E943D060E944C060E946B060E9472
:100D30007C067894CF91089583B7E82FFF27E7705A
:100D4000F070EE0FFF1FEF5FFE4F859194910895B5
:100D50008EB5E82FFF27E770F070EE0FFF1FEF5FF3
:100D6000FE4F85919491089585B5E82FFF27E77090
:100D7000F070EE0FFF1FEF5FFE4F85919491089585
:100D800080918A00E82FFF27E770F070EE0FFF1FB9
:100D9000EF5FFE4F8591949108958E3040F4E82FD7
:100DA000FF27EE0FFF1FEB5BFE4F608371830895FB
:100DB0000895DF92EF92FF920F931F93CF93DF93EB
:100DC000EC01D4B410921307109214071092150777
:100DD000109216070E94B4069C014427552760E034
:100DE00074E284EF90E00E94921C293B8DE8380762
:100DF00086E0480780E05807C0F487E2C131D80791
:100E0000A0F4CE01AA27BB27BC01CD010E943D1C46
:100E1000DC01CB01BC01CD0128EE33E040E050E025
:100E20000E94701CFA01E90111C07E010027112700
:100E3000CA01B90128EE33E040E050E00E94701C86
:100E4000C801B7010E943D1CFC01EB018091130712
:100E500090911407A0911507B09116072227382FFB
:100E6000492F5A2F84B59927AA27BB27282B392B1E
:100E70004A2B5B2BCD0DD11DE11DF11D2C173D071C
:100E80004E075F0758F58091130790911407A091C2
:100E90001507B091160785B7837E85BF85B7806239
:100EA00085BF889585B78F7D85BF80911307909109
:100EB0001407A0911507B0911607BA2FA92F982FE4
:100EC000882724B5332744275527822B932BA42B1F
:100ED000B52B8C179D07AE07BF07A8F2DF91CF9106
:100EE0001F910F91FF90EF90DF90089580910B0775
:100EF00090910C07A0910D07B0910E07BC01CD0198
:100F000008958091170790911807A0911907B09143
:100F10001A07BC01CD010895893031F48FB5826084
:100F20008FBD8FB58E7F0AC08A3019F48FB582606D
:100F300002C08FB58D7F8FBD8FB581608FBD1BBC0B
:100F40001ABC19BC18BC1092790010927800089550
:100F50009C018FB58E7F8FBD8FB582608FBD8EB5A2
:100F600088608EBD8EB580618EBD832F992787BD29
:100F700026BD1BBC1ABC19BC18BC1092790010927B
:100F8000780008958FB58F778FBD8FB58F7B8FBD1C
:100F900008958FB58F7D8FBD8FB58F7E8FBD0895DE
:100FA0008FB5877F8FBD8FB58B7F8FBD08958FB530
:100FB0008D7F8FBD8FB58E7F8FBD0E94C2070E942F
:100FC000C9070E94D00708958FB580688FBD8FB57F
:100FD0008F7B8FBD08958FB580628FBD8FB58F7E5B
:100FE0008FBD08958FB588608FBD8FB58B7F8FBD06
:100FF00008959C01892F99278BBD2ABD08959C01D6
:10100000892F992789BD28BD08959C01892F99278B
:1010100080937900209378000895893049F4809175
:101020008B00826080938B0080918B008E7F0EC03E
:101030008A3021F480918B00826003C080918B0004
:101040008D7F80938B0080918B00816080938B00DB
:1010500010928700109286001092850010928400F2
:10106000109283001092820008959C0180918B0061
:101070008E7F80938B0080918B00826080938B00A9
:1010800080918A00886080938A0080918A008061C4
:1010900080938A00832F992780938100209380007A
:1010A00010928700109286001092850010928400A2
:1010B0001092830010928200089580918B008F77A8
:1010C00080938B0080918B008F7B80938B000895A1
:1010D00080918B008F7D80938B0080918B008F7E21
:1010E00080938B00089580918B00877F80938B0085
:1010F00080918B008B7F80938B00089580918B0073
:101100008D7F80938B0080918B008E7F80938B00EE
:101110000E945D080E9468080E94730808958091EB
:101120008B00806880938B0080918B008F7B8093F5
:101130008B00089580918B00806280938B0080915A
:101140008B008F7E80938B00089580918B00886048
:1011500080938B0080918B008B7F80938B00089510
:101160009C01892F992780938700209386000895FA
:101170009C01892F992780938500209384000895EE
:101180009C01832F992780938300209382000895E8
:101190001F920F920FB60F9211242F933F934F93EC
:1011A0005F936F937F938F939F93AF93BF93EF93CF
:1011B000FF9380910B0790910C07A0910D07B091C0
:1011C0000E070196A11DB11D80930B0790930C078C
:1011D000A0930D07B0930E0780910B0790910C0719
:1011E000A0910D07B0910E070097A105B10599F4E4
:1011F00080911B0790911C07A0911D07B0911E07BD
:101200000196A11DB11D80931B0790931C07A0930D
:101210001D07B0931E078091450190914601892BCF
:1012200029F0E0914501F09146010995FF91EF9178
:10123000BF91AF919F918F917F916F915F914F91EE
:101240003F912F910F900FBE0F901F9018951F92F6
:101250000F920FB60F9211242F933F934F935F93EA
:101260006F937F938F939F93AF93BF93EF93FF936E
:101270008091490190914A01892B29F0E09149011F
:10128000F0914A010995FF91EF91BF91AF919F9124
:101290008F917F916F915F914F913F912F910F901F
:1012A0000FBE0F901F9018951F920F920FB60F92BE
:1012B00011242F933F934F935F936F937F938F935B
:1012C0009F93AF93BF93EF93FF93809117079091F4
:1012D0001807A0911907B0911A070196A11DB11D19
:1012E0008093170790931807A0931907B0931A07D4
:1012F0008091170790911807A0911907B0911A07CC
:101300000097A105B10599F480910F0790911007FE
:10131000A0911107B09112070196A11DB11D8093F4
:101320000F0790931007A0931107B09312078091B5
:10133000130790911407A0911507B0911607019615
:10134000A11DB11D8093130790931407A093150757
:10135000B09316078091530190915401892B29F085
:10136000E0915301F09154010995FF91EF91BF91E4
:10137000AF919F918F917F916F915F914F913F912D
:101380002F910F900FBE0F901F9018951F920F92E4
:101390000FB60F9211242F933F934F935F936F9348
:1013A0007F938F939F93AF93BF93EF93FF9380911E
:1013B000570190915801892B29F0E0915701F09144
:1013C00058010995FF91EF91BF91AF919F918F9136
:1013D0007F916F915F914F913F912F910F900FBE31
:1013E0000F901F9018951F920F920FB60F92112415
:1013F0002F933F934F935F936F937F938F939F931D
:10140000AF93BF93EF93FF93809147019091480171
:10141000892B29F0E0914701F09148010995FF914E
:10142000EF91BF91AF919F918F917F916F915F915C
:101430004F913F912F910F900FBE0F901F901895D5
:101440001F920F920FB60F9211242F933F934F9339
:101450005F936F937F938F939F93AF93BF93EF931C
:10146000FF9380914B0190914C01892B29F0E091E1
:101470004B01F0914C010995FF91EF91BF91AF9114
:101480009F918F917F916F915F914F913F912F919C
:101490000F900FBE0F901F9018951F920F920FB6CE
:1014A0000F9211242F933F934F935F936F937F93EA
:1014B0008F939F93AF93BF93EF93FF9380914D01D1
:1014C00090914E01892B29F0E0914D01F0914E0150
:1014D0000995FF91EF91BF91AF919F918F917F916E
:1014E0006F915F914F913F912F910F900FBE0F9091
:1014F0001F9018951F920F920FB60F9211242F93E1
:101500003F934F935F936F937F938F939F93AF938B
:10151000BF93EF93FF9380914F0190915001892BDE
:1015200029F0E0914F01F09150010995FF91EF9161
:10153000BF91AF919F918F917F916F915F914F91EB
:101540003F912F910F900FBE0F901F9018951F92F3
:101550000F920FB60F9211242F933F934F935F93E7
:101560006F937F938F939F93AF93BF93EF93FF936B
:101570008091510190915201892B29F0E091510104
:10158000F09152010995FF91EF91BF91AF919F9119
:101590008F917F916F915F914F913F912F910F901C
:1015A0000FBE0F901F9018951F920F920FB60F92BB
:1015B00011242F933F934F935F936F937F938F9358
:1015C0009F93AF93BF93EF93FF93809155019091B9
:1015D0005601892B29F0E0915501F09156010995AA
:1015E000FF91EF91BF91AF919F918F917F916F91FB
:1015F0005F914F913F912F910F900FBE0F901F90D1
:1016000018951F920F920FB60F9211242F933F93AC
:101610004F935F936F937F938F939F93AF93BF93FA
:10162000EF93FF938091590190915A01892B29F0F2
:10163000E0915901F0915A010995FF91EF91BF9105
:10164000AF919F918F917F916F915F914F913F915A
:101650002F910F900FBE0F901F9018951F920F9211
:101660000FB60F9211242F933F934F935F936F9375
:101670007F938F939F93AF93BF93EF93FF9380914B
:101680005B0190915C01892B29F0E0915B01F09165
:101690005C010995FF91EF91BF91AF919F918F915F
:1016A0007F916F915F914F913F912F910F900FBE5E
:1016B0000F901F9018951F920F920FB60F92112442
:1016C0002F933F934F935F936F937F938F939F934A
:1016D000AF93BF93EF93FF9380915D0190915E0173
:1016E000892B29F0E0915D01F0915E010995FF9150
:1016F000EF91BF91AF919F918F917F916F915F918A
:101700004F913F912F910F900FBE0F901F90189502
:101710001F920F920FB60F9211242F933F934F9366
:101720005F936F937F938F939F93AF93BF93EF9349
:10173000FF9380915F0190916001892B29F0E091E6
:101740005F01F09160010995FF91EF91BF91AF9119
:101750009F918F917F916F915F914F913F912F91C9
:101760000F900FBE0F901F901895209171002E7F43
:1017700020937100209171002D7F209371009C01B6
:101780004427552760E87EE380E090E00E94921CA9
:10179000DA01C901203148F03327C901409797FF8A
:1017A00002C0C9010F9795958795809370000895A1
:1017B0001092A9011092A8011092AB011092AA01F7
:1017C00084E690E00E94B50B809174008460809361
:1017D0007400109262011092610180917400816026
:1017E0008093740080917400806480937400789476
:1017F00008951092A9011092A8011092AB011092C5
:10180000AA0184E690E00E94B50B85E48093740001
:1018100078940895282F33272E7F3070611121602E
:101820002093720008959093A9018093A8010895D0
:101830009093AB018093AA010895809174008F70FA
:10184000806A809374000895809174008F70806D19
:10185000809374000895809174008823E4F70895BC
:1018600080937300809174008F70806880937400FF
:101870000895882329F0809174008F70806C04C0D3
:10188000809174008F70806880937400089508952B
:101890008091730099270895809171009927089588
:1018A000282FDA018091610190916201892BD1F793
:1018B00082E090E090936201809361012E7F2093FB
:1018C0006301662339F0E4E6F1E0962F8D91819370
:1018D0009150E1F71092840160938501809174002A
:1018E0008F70806A809374000895282FDA018091A8
:1018F000610190916201892BD1F783E090E0909390
:101900006201809361012160209363011092A6011E
:101910006093A701809174008F70806A8093740037
:101920008091610190916201892BD1F7662331F09A
:10193000E6E8F1E081918D936150E1F70895282F59
:10194000FA0190E0809174008E7F80937400809102
:1019500074008F70806A8093740080917400882373
:10196000E4F72E7F20937300809174008F7080685D
:1019700080937400809174008823E4F78091710053
:10198000883189F4662381F081918093730080917E
:1019900074008F7080688093740080917400882335
:1019A000E4F76150EFCF91E0809174008F70806D0B
:1019B000809374008091740084FFFCCF8091740048
:1019C000816080937400892F99270895282FDA0168
:1019D00090E0809174008E7F8093740080917400F9
:1019E0008F70806A80937400809174008823E4F77C
:1019F000216020937300809174008F7080688093C1
:101A00007400809174008823E4F780917100803421
:101A100009F5623088F0809174008F70806C80933B
:101A20007400809174008823E4F780917300FD01B5
:101A3000119680836150EDCF809174008F70806823
:101A400080937400809174008823E4F78091730080
:101A50008C9301C091E0809174008F70806D8093B1
:101A6000740080917400816080937400892F99279D
:101A700008951F920F920FB60F9211242F933F9348
:101A80004F935F936F937F938F939F93AF93BF9386
:101A9000EF93FF9380917100887F282F33272036A2
:101AA000310509F4D0C0213631050CF041C028328F
:101AB000310509F489C029323105CCF420313105D2
:101AC00009F47FC0213131054CF42115310509F4A9
:101AD0001FC12830310509F474C024C128313105F3
:101AE00009F472C02032310509F48BC01BC12034C7
:101AF000310509F49CC0213431054CF42033310503
:101B000009F47FC02833310509F480C00BC12035AA
:101B1000310509F480C0213531052CF42834310514
:101B200009F46FC0FFC02835310509F45EC0FAC062
:101B30002839310509F4DAC0293931050CF528377F
:101B4000310509F480C0293731054CF428363105B8
:101B500009F479C02037310509F475C0E3C028388D
:101B6000310509F4C3C0293831052CF4203831057A
:101B700009F476C0D7C02039310509F471C0D2C04C
:101B8000203B310509F48DC0213B31054CF4203A4E
:101B9000310509F474C0283A310509F482C0C2C085
:101BA000203C310509F4A9C0213C31052CF4283B27
:101BB000310509F48AC0B6C0283C310509F49DC03E
:101BC000B1C0809163010EC0909184018091850124
:101BD0009817B8F4E92FFF27EC59FE4F9F5F9093B9
:101BE000840180818093730081C08091A601E82FD9
:101BF000FF27EA57FE4F9091730090838F5F809389
:101C0000A601809174008F70806D7BC080917400FC
:101C10008F70806876C08091A601E82FFF27EA5771
:101C2000FE4F9091730090838F5F8093A601809107
:101C3000A601282F33278091A701992701972817FC
:101C400039074CF053C085E090E090936201809397
:101C500061011092A601809174008F70806C4AC05F
:101C60008091A601E82FFF27EA57FE4F909173005D
:101C700090838F5F8093A601803268F337C0809194
:101C800074008F70806C80937400E091A801F091D3
:101C9000A9013097C1F166E871E08091A60109952C
:101CA00032C084E090E09093620180936101E09102
:101CB000AA01F091AB01309731F064E671E080E267
:101CC0000995809385011092840190918401E92FF8
:101CD000FF27EC59FE4F9F5F909384018081809392
:101CE000730080918501981708F4B5CF8091740036
:101CF0008F7080688093740015C0809174008F701D
:101D0000806C8093740010926201109261010AC08D
:101D1000809174008F70806D8093740030936201A5
:101D200020936101FF91EF91BF91AF919F918F91AE
:101D30007F916F915F914F913F912F910F900FBEC7
:101D40000F901F9018958091610190916201089504
:101D50001F93182FDB01CA0173E0880F991FAA1F78
:101D6000BB1F7A95D1F79C01AD01220F331F441F91
:101D7000551F80509C4DAB40BF4FBC01CD010E9410
:101D8000701CDA01C9010197292F3327112329F08B
:101D9000809399002093980003C089B92093900004
:101DA0001F91089540E052E06CEA74E089E297E008
:101DB0000E94531140E450E06CEA76E08BE397E038
:101DC0000E94531108950E94D20E1092EF061092B5
:101DD000EE0688ED80939A0040E855E260E070E0FE
:101DE00081E00E94A80E8FEF8093200710923207A7
:101DF00010924607109245077894089540E052E00B
:101E00006CEA71E081E297E00E94531140E051E0FA
:101E10006CEA73E083E397E00E94531108950E94F7
:101E2000FE0E1092ED061092EC0688ED8AB940E89D
:101E300055E260E070E080E00E94A80E8FEF809392
:101E40001F071092310710924407109243077894AD
:101E500008950E940F0F0E94E30E0895823040F40F
:101E6000E82FFF27EE0FFF1FE451F94F60837183C6
:101E7000089508959927E3E0880F991FEA95E1F7FF
:101E80008F5D984F08959927F3E0880F991FFA9571
:101E9000E1F78D5C984F0895982FE82FFF27DF0119
:101EA000A15EB84F8C918823E9F3992319F06093D0
:101EB0009C0001C06CB9E15EF84F10820895682F54
:101EC00080E00E944C0F0895682F81E00E944C0F23
:101ED0000895CF93DF93EB01E82FFF27A3E0EE0FE8
:101EE000FF1FAA95E1F7EF5DF84F8281938100977C
:101EF00051F084819581009731F0CF010E945D11EE
:101F000088838FEF90E0DF91CF910895CF93DF9397
:101F1000CDB7DEB721970FB6F894DEBF0FBECDBFA9
:101F2000BE016F5F7F4F81E00E94690F882319F027
:101F30008981992702C08FEF9FEF21960FB6F89401
:101F4000DEBF0FBECDBFDF91CF910895CF93DF935A
:101F5000CDB7DEB721970FB6F894DEBF0FBECDBF69
:101F6000BE016F5F7F4F80E00E94690F882319F0E8
:101F70008981992702C08FEF9FEF21960FB6F894C1
:101F8000DEBF0FBECDBFDF91CF9108959927B3E09B
:101F9000880F991FBA95E1F78F5D984F0E94E7115E
:101FA000089520E030E0E82FFF2783E0EE0FFF1FC9
:101FB0008A95E1F7EF5DF84F84819581892B11F4C3
:101FC00021E030E0C9010895992733E0880F991F77
:101FD0003A95E1F78D5C984F0E94B6110895682FED
:101FE00080E00E94E40F0895682F81E00E94E40FD2
:101FF00008951F93182F9927FC01EF5CF84F2FEFDE
:10200000208343E0880F991F4A95E1F78D5C984F34
:102010000E945D11682F812F0E944C0F1F9108951F
:10202000CF92DF92EF92FF920F931F93CF93DF93A4
:10203000D82E8B01E82EFF24F70163E0EE0FFF1F7F
:102040006A95E1F7ED5CF84F84819581840F951FC7
:10205000228133818217930740F54115510529F1FB
:10206000F801C1908F014130510591F0EA012197AB
:10207000F80121918F01C70153E0880F991F5A95EC
:10208000E1F7622F8D5C984F0E94B611219781F77E
:10209000ED2DFF27EF5CF84F8FEF80836C2D8D2D9A
:1020A0000E944C0F8FEF90E002C080E090E0DF9143
:1020B000CF911F910F91FF90EF90DF90CF900895F7
:1020C000CF93DF93282FA82FBB27ED01CF5CD84FEC
:1020D00088818823E1F0FD0173E0EE0FFF1F7A9500
:1020E000E1F7ED5CF84F84819581892B79F022230B
:1020F00039F08BE397E00E945D1180939C000BC048
:1021000083E397E00E945D118CB905C01882A15E3F
:10211000B84F8FEF8C93DF91CF910895CF93DF93DA
:10212000882319F060919C0001C06CB1282F3327DF
:10213000E901C20FD31FFE01E451F94F8081918163
:10214000892B31F00190F081E02D862F099514C084
:10215000E3E0220F331FEA95E1F7C9018F5D984F45
:102160000E94B611882341F4FE01ED5BF84F808197
:102170009181019680839183DF91CF9108951F9281
:102180000F920FB60F9211242F933F934F935F93AB
:102190006F937F938F939F93AF93BF93EF93FF932F
:1021A00080E00E946010FF91EF91BF91AF919F91ED
:1021B0008F917F916F915F914F913F912F910F90F0
:1021C0000FBE0F901F9018951F920F920FB60F928F
:1021D00011242F933F934F935F936F937F938F932C
:1021E0009F93AF93BF93EF93FF9381E00E946010A2
:1021F000FF91EF91BF91AF919F918F917F916F91DF
:102200005F914F913F912F910F900FBE0F901F90B4
:1022100018951F920F920FB60F9211242F933F9390
:102220004F935F936F937F938F939F93AF93BF93DE
:10223000EF93FF9380E00E948E10FF91EF91BF918A
:10224000AF919F918F917F916F915F914F913F914E
:102250002F910F900FBE0F901F9018951F920F9205
:102260000FB60F9211242F933F934F935F936F9369
:102270007F938F939F93AF93BF93EF93FF9381E0EF
:102280000E948E10FF91EF91BF91AF919F918F911E
:102290007F916F915F914F913F912F910F900FBE62
:1022A0000F901F901895FC016083718342835383C4
:1022B00016821782148215820895CF93DF93EC0162
:1022C000E0E02C813D8121153105B9F08E819F819F
:1022D000E881F981E80FF91FE08101968E839F83E1
:1022E0006A817B818617970720F00E945C1C8E8391
:1022F0009F83215030402C833D838E2F9927DF917F
:10230000CF910895CF93DF93FC01EB0124813581B8
:1023100062177307A0F486819781860F971F8683C3
:102320009783628173818617970720F00E945C1C57
:10233000868397832C1B3D0B2483358302C0148234
:102340001582DF91CF910895FC01868197812281CA
:102350003381860F971FB9010E945C1C0190F081A8
:10236000E02DE80FF91F808199270895CF93DF931F
:10237000EC01462F2C813D816A817B81261737072E
:1023800098F48E819F81820F931F0E945C1CE881CC
:10239000F981E80FF91F40838C819D8101968C8320
:1023A0009D838FEF90E002C080E090E0DF91CF91BD
:1023B0000895FC0140E050E02481358182819381C1
:1023C0002817390710F441E050E0CA010895FC01D4
:1023D0001482158208959093F1068093F006089573
:1023E000E091F006F091F10609950895CF93DF93FF
:1023F000EC01892B61F08881882349F0E091F00697
:10240000F091F1068991099588818823B9F7DF91C8
:10241000CF910895EF92FF920F931F93CF93DF9385
:10242000EC017A0120E030E0892B01F1C9012F5F36
:102430003F4F8617970718F489918823B9F720E052
:1024400030E02E153F0590F4888189010F5F1F4F02
:10245000E091F006F091F106882311F0219601C079
:1024600080E2099598010E151F0570F3DF91CF9159
:102470001F910F91FF90EF900895CF93DF93EC01A0
:10248000009779F0FC0121968491882351F0E09126
:10249000F006F091F1060995FE01219684918823BA
:1024A000B1F7DF91CF910895E091F006F091F10638
:1024B0008DE00995E091F006F091F1068AE009952A
:1024C0000895E82FFF27EF70F070E35FFE4F8491CF
:1024D000E091F006F091F106099508951F93182FE9
:1024E00082958F700E946112812F0E9461121F914C
:1024F00008950F931F938C01812F99270E946E12CC
:10250000802F0E946E121F910F910895EF92FF92FB
:102510000F931F937B018C01C801AA27BB270E9440
:102520007912C7010E9479121F910F91FF90EF90CD
:1025300008952F923F924F925F926F927F928F9267
:102540009F92AF92BF92CF92DF92EF92FF920F9342
:102550001F93CF93DF93CDB7DEB7A2970FB6F89452
:10256000DEBF0FBECDBF69A3C42E2AA32701380149
:10257000442351F017FF08C0EE24FF248701E4181C
:10258000F5080609170902C08301720199A1692F94
:10259000772767FD709561507040CC2011F0615035
:1025A0007040D62E18A22FE1222E312C2C0E3D1E6B
:1025B000882E992487FC9094A92CB92CC801B701C6
:1025C000A50194010E94701CDC01CB01FC01E35FBA
:1025D000FE4F84918F8FC801B701A50194010E941D
:1025E000701C79018A01DA94AFEFDA1639F1DA94C6
:1025F000C1010197E114F10401051105C1F01C01AD
:10260000C801B701A50194010E94701CDC01CB0137
:10261000FC01E35FFE4F8491F1018083C801B701A3
:10262000A50194010E94701C79018A0104C01C015B
:10263000EAA1DC01EC93FFEFDF16C9F6CC20B9F07C
:1026400077FE05C08DE2D1018E931D0110C0C1013E
:10265000019714141504160417042CF41C018BE2C2
:10266000F101808304C01C0180E2D1018C93D9A0C8
:10267000DA94BFEFDB1661F0E091F006F091F1061D
:10268000D1018D911D010995DA94BFEFDB16A1F7F9
:10269000A2960FB6F894DEBF0FBECDBFDF91CF91EB
:1026A0001F910F91FF90EF90DF90CF90BF90AF9070
:1026B0009F908F907F906F905F904F903F902F9062
:1026C00008957F928F929F92AF92BF92CF92DF92A6
:1026D000EF92FF920F931F93CF93DF93CDB7DEB7A7
:1026E0007888C988DA8863E1A62EB12CAC0EBD1EAD
:1026F00008C0882309F481C0E091F006F091F1064A
:10270000099596012F5F3F4F772021F0F60169016F
:10271000849103C0F60180816901853251F72F5FF2
:102720003F4F772021F0F6016901849103C0F60143
:1027300080816901282F332727FD30952436310504
:1027400091F02536310524F42336310529F0D4CF14
:102750002837310581F0D0CFF50122E030E0A20E1C
:10276000B31E8081C9CF5AE0852E912C40E1E42E22
:1027700047E2F42E04C030E1E32EF12C4701F501CD
:1027800022E030E0A20EB31E008111818436D9F41C
:1027900017FF09C0109501951F4FE091F006F091C9
:1027A000F1068DE2099532E0E316F10460F00E15B2
:1027B0001F0548F4C7016AE070E00E945C1C7B01C1
:1027C00062307105A0F7C801B7010E945C1CFB01D3
:1027D000E35FFE4F8491E091F006F091F1060995D8
:1027E000C801B7010E945C1C8C01C701B4010E94A2
:1027F0005C1C7B01672B39F784CF80E090E0DF9190
:10280000CF911F910F91FF90EF90DF90CF90BF90ED
:10281000AF909F908F907F900895811188E0809372
:10282000470708950895EF92FF921F93CF93DF9388
:10283000CDB7DEB721970FB6F894DEBF0FBECDBF80
:10284000182F80E8898380E00E940D14EE24FF2475
:10285000AE014F5F5F4F61E0812F0E949F0C882384
:1028600019F481E0E82EF12CC70121960FB6F894F7
:10287000DEBF0FBECDBFDF91CF911F91FF90EF90D4
:1028800008951F93CF93DF93CDB7DEB723970FB68D
:10289000F894DEBF0FBECDBF182F862F807F90919A
:1028A0004707892B8983AE014F5F5F4F61E0812F1E
:1028B0000E949F0CAE014E5F5F4F62E0812F0E942D
:1028C000E60C8A819927382F22278B819927822B22
:1028D000932B23960FB6F894DEBF0FBECDBFDF91CA
:1028E000CF911F910895962F97709295907F692FA1
:1028F0000E9441140895962F9695492F5527262F0B
:10290000332721703070220F331F220F331F422BC9
:10291000532B34E0440F551F3A95E1F7642F60685C
:102920000E94411408951092F4061092F30610923A
:10293000490710924807EAE4F7E089E011928150D4
:1029400087FFFCCF109254070E940F0F40E659E01A
:1029500060E070E080E00E94A80E129A1A98089534
:10296000282F8091490799278130910589F082307D
:1029700091051CF4892B21F02BC00297C9F028C0C7
:102980002A3041F581E08093490710924807089565
:1029900080914807E82FFF27E65BF84F20838F5F81
:1029A000809348078A30B0F082E080934907089509
:1029B0002D3059F4E091F306F091F406309729F0A8
:1029C0006AE477E08091F20609951092490708952C
:1029D0001092490708950895CF93DF93CDB7DEB7DE
:1029E00021970FB6F894DEBF0FBECDBFBE016F5F5B
:1029F0007F4F80E00E94690F882319F089810E942F
:102A0000B01421960FB6F894DEBF0FBECDBFDF9194
:102A1000CF9108959093F4068093F306089530E2E1
:102A2000309368071092670730936A078EE191E050
:102A300090936C0780936B0782E280936E071092ED
:102A40006D073093700784E291E090937207809352
:102A5000710784E2809374071092730730937607AE
:102A60008AE291E0909378078093770786E28093DB
:102A7000AA071092A9073093AC0780E391E09093E6
:102A8000AE078093AD0788E28093B6071092B50732
:102A90003093B80786E391E09093BA078093B90723
:102AA0008AE28093BC071092BB073093BE078CE389
:102AB00091E09093C0078093BF078CE28093C20798
:102AC0001092C1073093C40782E491E09093C60747
:102AD0008093C5078EE28093C8071092C707309392
:102AE000CA0788E491E09093CC078093CB0784E3F6
:102AF00080937A071092790730937C078EE491E0F7
:102B000090937E0780937D0780E6809380071092E4
:102B10007F073093820784E591E090938407809348
:102B2000830780E780938607109285073093880794
:102B30008AE591E090938A078093890720E92093A2
:102B40008C0710928B0720938E0780E691E090937C
:102B5000900780938F07209392071092910740EA85
:102B60004093940789E691E09093960780939507A8
:102B7000209398071092970780EC80939A0782E73A
:102B800091E090939C0780939B0788E880939E0731
:102B900010929D073093A0078BE791E09093A207D6
:102BA0008093A10783E98093A4071092A307109252
:102BB000A60781E891E09093A8078093A70780E893
:102BC0008093B0071092AF073093B20787E891E087
:102BD0009093B4078093B3074093DA071092D90714
:102BE0003093DC078DE891E09093DE078093DD075A
:102BF00082E68093CE071092CD073093D00783E909
:102C000091E09093D2078093D10782E78093D40715
:102C10001092D3073093D60789E991E09093D807B3
:102C20008093D70784E68093E6071092E5073093F8
:102C3000E8078FE991E09093EA078093E90784E73A
:102C40008093E0071092DF073093E20785EA91E076
:102C50009093E4078093E30786E68093F20710924F
:102C6000F1073093F4078BEA91E09093F607809395
:102C7000F50786E78093EC071092EB073093EE0799
:102C800081EB91E09093F0078093EF0782E88093C7
:102C9000F8071092F7073093FA0787EB91E09093CB
:102CA000FC078093FB0784E88093FE071092FD07E2
:102CB000309300088DEB91E0909302088093010817
:102CC00080E480930408109203082FEF20930608F5
:102CD00083EC91E0909308088093070882E4809346
:102CE000100810920F082093120889EC91E090933D
:102CF00014088093130884E4809316081092150832
:102D0000209318088FEC91E090931A08809319088B
:102D100086E480931C0810921B0820931E0885ED02
:102D200091E09093200880931F0888E48093220804
:102D300010922108209324088BED91E090932608AF
:102D4000809325088AE4809328081092270820930E
:102D50002A0881EE91E090932C0880932B088AE852
:102D600080930A081092090820930C0887EE91E0DE
:102D700090930E0880930D080895CF93DF93CDB7FD
:102D8000DEB721970FB6F894DEBF0FBECDBF6983C3
:102D90009927FC01EE0FFF1FEE0FFF1FE80FF91F31
:102DA000E80FF91FED5FF74FAE014F5F5F4F61E036
:102DB00081810E949F0C992721960FB6F894DEBF5F
:102DC0000FBECDBFDF91CF9108951F93CF93DF93B7
:102DD00013B3C12FDD279E012170307080916607EB
:102DE0009927817090702817390781F081E090E071
:102DF0008C279D27AA27BB2781709070A070B07088
:102E0000AC01BD018FEE91E00E94A4039E012270EF
:102E10003070809166079927827090702817390763
:102E200099F0CE019695879521E030E0822793278F
:102E3000AA27BB2781709070A070B070AC01BD0153
:102E400084EF91E00E94A4039E0124703070809171
:102E5000660799278470907028173907A9F0CE016A
:102E6000969587959695879521E030E08227932760
:102E7000AA27BB2781709070A070B070AC01BD0113
:102E800089EF91E00E94A4039E0128703070809128
:102E9000660799278870907028173907B1F0CE011E
:102EA00073E0969587957A95E1F721E030E08227E7
:102EB0009327AA27BB2781709070A070B070AC01D7
:102EC000BD018EEF91E00E94A4039E01207130703D
:102ED0008091660799278071907028173907B1F0A3
:102EE000CE0164E0969587956A95E1F721E030E0A0
:102EF00082279327AA27BB2781709070A070B0709B
:102F0000AC01BD0183E092E00E94A4039E01207207
:102F10003070809166079927807290702817390762
:102F2000B1F0CE0155E0969587955A95E1F721E0ED
:102F300030E082279327AA27BB2781709070A0706A
:102F4000B070AC01BD0188E092E00E94A4039E0134
:102F500020743070809166079927807490702817CC
:102F60003907B1F0CE0146E0969587954A95E1F78D
:102F700021E030E082279327AA27BB278170907039
:102F8000A070B070AC01BD018DE092E00E94A4037E
:102F9000C078D07080916607992780789070C817A4
:102FA000D907B1F0812F992787FD9095A92FB92FC7
:102FB00080959095A095B0958827B7FD8395992722
:102FC000AA27BB27AC01BD0182E192E00E94A403C5
:102FD00010936607DF91CF911F9108959927FC0107
:102FE000EE0FFF1FEE0FFF1FE80FF91FE80FF91F8D
:102FF000E959F84F82819927AA27BB27AC01BD0167
:10300000848195810E94A403089580916500816068
:103010008093650085E090E00E94D906809165006C
:103020008E7F809365000895DF92EF92FF920F9359
:103030001F93CF93DF93CDB7DEB723970FB6F894E6
:10304000DEBF0FBECDBFD82E86E0D89EC0011124B2
:103050008659984FED2CFF248701000F111F000F98
:10306000111F0E0D1F1D0E0D1F1D0959184FAC010C
:1030700061E0F80181810E949F0C84E690E00E944B
:103080000706C70106970397C0F4AE014F5F5F4F75
:1030900062E0F80181810E94E60C482F898199271E
:1030A000982F88272A813327822B932B24E095950C
:1030B00087952A95E1F78B8309C0AE014D5F5F4F7D
:1030C00061E0F80181810E94E60C482F413021F433
:1030D0008D2D0E94051840C0F701EE0FFF1FEE0F67
:1030E000FF1FEE0DFF1DEE0DFF1DE959F84F2B815F
:1030F0008281281789F1F3E1EF16F1044CF481E1A4
:10310000E816F1044CF4C70104970297B0F404C028
:10311000C7014497049788F4F701EE0FFF1FEE0FE5
:10312000FF1FEE0DFF1DEE0DFF1DE959F84F8281C7
:10313000821B885F813160F40FC0F701EE0FFF1F23
:10314000EE0FFF1FEE0DFF1DEE0DFF1DE959F84FAD
:10315000228381E090E002C080E090E023960FB6E9
:10316000F894DEBF0FBECDBFDF91CF911F910F91BD
:10317000FF90EF90DF9008951F93CF93DF9310E0BF
:1031800086E0189F900111242659384F812F9927E6
:10319000EC01CC0FDD1FCC0FDD1FC80FD91FC80FEE
:1031A000D91FC959D84FA90161E089810E949F0C9C
:1031B00098811F5F813051F4992331F06C817D81BA
:1031C00087E192E00E94D40218820AC0992331F468
:1031D0006C817D8183E292E00E94D40281E0888349
:1031E0001A3170F210E086E0189F900111242A5FD6
:1031F000374F812F9927EC01CC0FDD1FCC0FDD1F3E
:10320000C80FD91FC80FD91FCD5FD74FA90161E0E3
:1032100089810E949F0C1F5F9881813051F499230E
:1032200031F06C817D818CE292E00E94D4021882A0
:103230000AC0992331F46C817D8188E392E00E9479
:10324000D40281E08883173070F2DF91CF911F9113
:1032500008958F929F92AF92BF92CF92DF92EF929A
:10326000FF921F93CF93DF934C015A016B0161E4EE
:1032700072E00E94251C009731F59C0119E1FC01C8
:10328000E20FF31FE959F84F108211502F5F3F4FA3
:10329000059617FFF4CF80E090E09C0116E0FC015A
:1032A000E20FF31FED5FF74F108211502F5F3F4F7A
:1032B000059617FFF4CF0E94BC181FC06A2D812FFE
:1032C0000E94BD161AC010E0C0E0D0E07E01FE01F1
:1032D000EE0DFF1DED5FF74F8081882339F064818B
:1032E0007581C4010E94251C892B41F31F5F08943E
:1032F000E11CF11C2596173050F3DF91CF911F91FF
:10330000FF90EF90DF90CF90BF90AF909F908F9005
:103310000895DF92EF92FF920F931F93CF93DF9365
:10332000EC017A018B01DD2444E050E069E472E0B5
:103330000E942F1C892BA9F5FE0101900020E9F7BE
:103340003697EC17FD0709F095C08C81803329F47E
:103350008E2D99270E94C0088DC0813329F48E2DAF
:1033600099270E94B80886C0823329F48E2D9927A8
:103370000E94B0087FC0833329F48E2D99270E94C4
:10338000050878C0843329F48E2D99270E94FF0701
:1033900071C0853309F06EC08E2D99270E94F90700
:1033A00069C044E050E06EE472E0CE010E942F1C40
:1033B000892B09F05FC0FE0101900020E9F73697E4
:1033C000EC17FD0709F056C08C81992787FD909571
:1033D00083339105F1F0843391054CF481339105E9
:1033E00091F08233910594F4C09709F143C085337D
:1033F0009105A9F0853391057CF08633910591F014
:10340000C79799F037C081E0D82E11C0C2E0DC2EFA
:103410000EC0B3E0DB2E0BC0A4E0DA2E08C0F5E04E
:10342000DF2E05C0E6E0DE2E02C077E0D72E81E079
:1034300090E0A0E0B0E0E822F9220A231B232D2D22
:103440003327EF2869F081E090E002C0880F991FD0
:103450002A95E2F7982F90958BB389238BBB0AC0EE
:1034600081E090E002C0880F991F2A95E2F72BB304
:10347000282B2BBBDF91CF911F910F91FF90EF90E5
:10348000DF9008951F93182F0E94C601382F9927A7
:10349000412F5527FA01EB5AF84F2081821B9109E1
:1034A0000896419708F467C0308343305105A9F16D
:1034B000443051054CF441305105E9F0423051059A
:1034C0001CF5452B79F057C045305105C1F1453009
:1034D000510564F146305105D9F14730510509F4E1
:1034E00040C049C0832F9927AA27BB27AC01BD0143
:1034F00083E592E03EC0832F9927AA27BB27AC0122
:10350000BD0189E592E035C0832F9927AA27BB2703
:10351000AC01BD018FE592E02CC0832F9927AA272B
:10352000BB27AC01BD0185E692E023C0832F99271C
:10353000AA27BB27AC01BD018BE692E01AC0832FFE
:103540009927AA27BB27AC01BD0181E792E011C0F2
:10355000832F9927AA27BB27AC01BD0187E792E0FB
:1035600008C0832F9927AA27BB27AC01BD018DE78F
:1035700092E00E94A4031F910895CEEFD0E1DEBF38
:10358000CDBF0E94890680E00E94051881E08093EB
:1035900064001092650014BA8FEF85BB8ABB1BBA1A
:1035A0000E949201BD9ABE9ABF9A139A149A159AD4
:1035B0000E944C0688E00E948C070E94E4070E944B
:1035C000EB070E94F20780E090E00E94F90780E09C
:1035D00090E00E94FF0780E090E00E9405080E94B2
:1035E0007C0688E00E940D080E948F080E949A08BD
:1035F0000E94A50880E090E00E94B00880E090E082
:103600000E94B80880E090E00E94C0080E940F0F5E
:1036100040E052EC61E070E080E00E94A80E0E9461
:10362000DD010E94010489E899E10E94210491E0F2
:10363000E92EF12C0E94E51610E0812F0E94421A1B
:103640001F5F1830D0F3BE016F5F7F4F80E00E9494
:10365000690F882319F089810E942604C7018170AF
:1036600090700894E11CF11C892B21F08091650079
:10367000816003C0809165008E7F80936500DACF02
:103680001F93CF93DF9313B3C12FDD279E012170CA
:10369000307080915D0799278170907028173907E5
:1036A00081F081E090E08C279D27AA27BB278170BD
:1036B0009070A070B070AC01BD0183E892E00E94F0
:1036C000A4039E012470307080915D079927847057
:1036D000907028173907A9F0CE0196958795969591
:1036E000879521E030E082279327AA27BB278170A6
:1036F0009070A070B070AC01BD0188E892E00E94AB
:10370000A4039E012071307080915D07992780711C
:10371000907028173907B1F0CE0134E0969587955F
:103720003A95E1F721E030E082279327AA27BB27CB
:1037300081709070A070B070AC01BD018DE892E016
:103740000E94A4039E012074307080915D07992728
:103750008074907028173907B1F026E0D695C79588
:103760002A95E1F781E090E0C827D927CE01AA2762
:10377000BB2781709070A070B070AC01BD0182E970
:1037800092E00E94A40310935D07DF91CF911F91F7
:10379000089599278130910579F0823091051CF4C4
:1037A000892B39F008958230910559F0039761F023
:1037B000089587E992E002C08EE992E00E94080332
:1037C000089585EA92E0FACF8CEA92E0F7CF1F9352
:1037D000182F0E94C601382F9927412F5527FA012B
:1037E000E25AF84F2081821B91090896419758F1BF
:1037F000308343305105A1F04430510524F4413069
:10380000510529F020C04530510599F01CC0832F87
:103810009927AA27BB27AC01BD0183EB92E011C019
:10382000832F9927AA27BB27AC01BD0189EB92E022
:1038300008C0832F9927AA27BB27AC01BD018FEBB6
:1038400092E00E94A4031F910895FB01DC018D9179
:103850000590801911F40020D1F7990B0895FB0110
:10386000DC014150504030F08D910590801919F4E1
:103870000020B9F7881B990B0895629FD001739FB0
:10388000F001829FE00DF11D649FE00DF11D929FFC
:10389000F00D839FF00D749FF00D659FF00D99273B
:1038A000729FB00DE11DF91F639FB00DE11DF91F5F
:1038B000BD01CF0111240895AA1BBB1B51E107C014
:1038C000AA1FBB1FA617B70710F0A61BB70B881FB0
:1038D000991F5A95A9F780959095BC01CD0108953F
:1038E000A1E21A2EAA1BBB1BFD010DC0AA1FBB1F04
:1038F000EE1FFF1FA217B307E407F50720F0A21B76
:10390000B30BE40BF50B661F771F881F991F1A94E2
:1039100069F760957095809590959B01AC01BD010C
:10392000CF01089597FB092E05260ED057FD04D030
:10393000D7DF0AD0001C38F450954095309521957A
:103940003F4F4F4F5F4F0895F6F7909580957095D4
:0A39500061957F4F8F4F9F4F089540
:02395A0001006A
:00000001FF
